:1000000027C441C440C43FC43EC43DC43CC43BC4F7
:100010003AC439C438C471C536C435C434C433C4D1
:1000200032C400003A00370000003B0038000101F4
:100030000101010101010202020102040810204035
:100040008004020100000000000403020100008F90
:10005000008E008D008D008C008B008A0089008846
:100060000088008700860085008500840083008268
:10007000008100810080007F007E007E007D007C8A
:10008000007C007B007A00790079007800770077A7
:1000900000760075007500740073007300720072C2
:1000A000007100700070006F006E006E006D006DDA
:1000B000006C006B006B006A006A006900690068F0
:1000C0000067006700660066006500650064006404
:1000D0000063006300620062006100610060006014
:1000E000005F005F005E005E005D005D005C005C24
:1000F000005C005B005B005A005A00590059005830
:10010000005800580057005700560056005600553A
:100110000055005400540054005300530052005244
:100120000052005100510051005000500050004F4B
:10013000004F004F004E004E004D004D004D004D51
:10014000004C004C004C004B004B004B004A004A56
:10015000004A004900490049004900480048004859
:10016000004700470047004700460046004600455C
:10017000004500450045004400440044004400435D
:10018000004300430043004200420042004200425C
:10019000004100410041004100400040004000405B
:1001A0000040003F003F003F003F003F003E003E58
:1001B000003E003E003E003D003D003D003D003D54
:1001C000003C003C003C003C003C003B003B003B52
:1001D000003B003B003B003A003A003A003A003A4C
:1001E000003A003900390039003900390039003847
:1001F0000038003800380038003800380037003741
:100200000037003700370037003700360036003639
:100210000036003600360036003500350035003532
:10022000003500350035003400340034003400342B
:100230000034003400340033003300330033003323
:10024000003300330033003300320032003200321A
:100250000032003200320032003200310031003111
:100260000031003100310031003100310030003008
:1002700000300030003000300030003000300030FE
:10028000002F002F002F002F002F002F002F002FF6
:10029000002F002F002E002E002E002E002E002EEC
:1002A000002E002E002E002E002D002D002D002DE2
:1002B000002D002D002D002D002D002D002D002CD7
:1002C000002C002C002C002C002C002C002C002CCE
:1002D000002C002C002B002B002B002B002B002BC4
:1002E000002B002B002B002B002B002A002A002AB9
:1002F000002A002A002A002A002A002A002A002AAE
:10030000002A0029002900290029002900290029A4
:100310000029002900290029002800280028002899
:10032000002800280028002800280028002800278E
:100330000027002700270027002700270027002785
:10034000002700270026002600260026002600267B
:10035000002600260026002600260026002500256F
:100360000025002500250025002500250025002565
:10037000002500240024002400240024002400245C
:100380000024002400240024002300230023002351
:100390000023002300230023002300230022002247
:1003A000002200220022002200220022002200223D
:1003B0000022002100210021002100210021002134
:1003C000002100210021002000200020002000202A
:1003D000002000200020002000200020001F001F1F
:1003E000001F001F001F001F001F001F001F001F15
:1003F000001E001E001E001E001E001E001E001E0D
:10040000001E001E001D001D001D001D001D001D02
:10041000001D001D001D001D001C001C001C001CF8
:10042000001C001C001C001C001C001C001B001BEE
:10043000001B001B001B001B001B001B001B001BE4
:10044000001A001A001A001A001A001A001A001ADC
:10045000001A001A001900190019001900190019D2
:1004600000190019001900190018001800180018C8
:1004700000180018001800180018001700170017BF
:1004800000170017001700170017001700170016B5
:1004900000160016001600160016001600160016AC
:1004A00000160015001500150015001500150015A3
:1004B0000015001500150014001400140014001499
:1004C000001400140014001400140013001300138F
:1004D0000013001300130013001300130012001286
:1004E000001200120012001200120012001200127C
:1004F0000011001100110011001100110011001174
:100500000011001100100010001000100010001069
:100510000010001000100010000F000F000F000F5F
:10052000000F000F000F000F000F000F000F000E54
:10053000000E000E000E000E000E000E000E000E4B
:10054000000E000D000D000D000D000D000D000D42
:10055000000D000D000D000C000C000C000C000C38
:10056000000C000C000C000C000C000C000B000B2D
:10057000000B000B000B000B000B000B000B000B23
:10058000000B000A000A000A000A000A000A000A1A
:10059000000A000A000A000A00090009000900090F
:1005A0000009000900090009000900090009000804
:1005B00000080008000800080008000800080008FB
:1005C00000080008000700070007000700070007F1
:1005D00000070007000700070007000700060006E5
:1005E00000060006000600060006000600060006DB
:1005F00000060005000500050005000500050005D2
:1006000000050005000500050005000400040004C5
:1006100000040004000400040004000400040004BA
:1006200000040003000300030003000300030003B1
:1006300000030003000300030002000200020002A6
:10064000000200020002000200020002000200029A
:100650000001000100010001000100010001000192
:100660000001000100010000000000000000000087
:1006700000000000000000000000000000FFFFFF7D
:10068000FFFFFFFFFFFFFFFFFFFFFFFFFFFFFFFF7A
:10069000FFFFFFFEFFFEFFFEFFFEFFFEFFFEFFFE71
:1006A000FFFEFFFEFFFEFFFDFFFDFFFDFFFDFFFD67
:1006B000FFFDFFFDFFFDFFFDFFFDFFFCFFFCFFFC5D
:1006C000FFFCFFFCFFFCFFFCFFFCFFFCFFFCFFFB53
:1006D000FFFBFFFBFFFBFFFBFFFBFFFBFFFBFFFA4B
:1006E000FFFAFFFAFFFAFFFAFFFAFFFAFFFAFFFA42
:1006F000FFF9FFF9FFF9FFF9FFF9FFF9FFF9FFF93A
:10070000FFF8FFF8FFF8FFF8FFF8FFF8FFF8FFF831
:10071000FFF7FFF7FFF7FFF7FFF7FFF7FFF7FFF62A
:10072000FFF6FFF6FFF6FFF6FFF6FFF6FFF5FFF523
:10073000FFF5FFF5FFF5FFF5FFF5FFF4FFF4FFF41C
:10074000FFF4FFF4FFF4FFF3FFF3FFF3FFF3FFF316
:10075000FFF3FFF2FFF2FFF2FFF2FFF2FFF1FFF112
:10076000FFF1FFF1FFF1FFF1FFF0FFF0FFF0FFF00D
:10077000FFF0FFEFFFEFFFEFFFEFFFEFFFEEFFEE0A
:10078000FFEEFFEEFFEEFFEDFFEDFFEDFFEDFFEC07
:10079000FFECFFECFFECFFECFFEBFFEBFFEBFFEB05
:1007A000FFEAFFEAFFEAFFEAFFE9FFE9FFE9FFE905
:1007B000FFE8FFE8FFE8FFE8FFE7FFE7FFE7FFE606
:1007C000FFE6FFE6FFE6FFE5FFE5FFE5FFE4FFE408
:1007D000FFE4FFE4FFE3FFE3FFE3FFE2FFE2FFE20A
:1007E000FFE1FFE1FFE1FFE0FFE0FFE0FFDFFFDF10
:1007F000FFDFFFDEFFDEFFDEFFDDFFDDFFDDFFDC15
:10080000FFDCFFDCFFDBFFDBFFDAFFDAFFDAFFD91B
:10081000FFD9FFD8FFD8FFD8FFD7FFD7FFD6FFD625
:10082000FFD6FFD5FFD5FFD4FFD4FFD3FFD3FFD32F
:10083000FFD2FFD2FFD1FFD1FFD0FFD0FFCFFFCF3C
:10084000FFCEFFCEFFCDFFCDFFCCFFCCFFCBFF0017
:1008500011241FBECFE5D2E0DEBFCDBF10E0A0E681
:10086000B0E0E8EFFFE002C005900D92AC36B107B2
:10087000D9F720E0ACE6B0E001C01D92AA37B2077C
:10088000E1F785D1B7C3BCCB90E0FC01EC5BFF4F37
:100890003491FC01E75CFF4F2491FC01E25DFF4FC6
:1008A000E491EE2351F13323B1F0323089F028F492
:1008B000313089F480B78F770DC0333029F0343070
:1008C00051F48FB58F7D02C08FB58F778FBD03C078
:1008D00080B78F7D80BFF0E0EE0FFF1FE85DFF4F18
:1008E000A591B4918FB7F894EC91611103C0209554
:1008F0002E2301C02E2B2C938FBF0895CF93DF930F
:1009000090E0FC01E75CFF4F2491FC01E25DFF4FAA
:100910008491882361F190E0880F991FFC01EE5DBE
:10092000FF4FC591D491FC01E85DFF4FA591B491B3
:10093000611109C09FB7F89488812095822388832C
:10094000EC912E230BC0623061F49FB7F89438818C
:10095000822F809583238883EC912E2B2C939FBF2D
:1009600006C08FB7F894E8812E2B28838FBFDF91C4
:10097000CF9108958E3008F08E5093B183FB2227DB
:1009800020F930E045E0220F331F4A95E1F79F7DC3
:10099000292B23B98770909175009295990F990F23
:1009A000907C892B87B9369A3699FECF84B125B1D0
:1009B00090E0922B08953FB7F89480917100909148
:1009C0007200A0917300B091740022B708B600FEC7
:1009D00005C02F3F19F00196A11DB11D3FBFBA2FD1
:1009E000A92F982F8827820F911DA11DB11DBC0131
:1009F000CD0146E0660F771F881F991F4A95D1F7F2
:100A000008958F929F92AF92BF92CF92DF92EF9212
:100A1000FF926B017C01CFDF4B015C01C114D1045B
:100A2000E104F104E9F0C7DFDC01CB018819990981
:100A3000AA09BB09883E9340A105B10578F321E0DE
:100A4000C21AD108E108F10888EE880E83E0981EEA
:100A5000A11CB11CC114D104E104F10421F7DECFC3
:100A6000FF90EF90DF90CF90BF90AF909F908F90CE
:100A700008950F931F93CF93DF93C7E0D0E0082F23
:100A800010E0B8010C2E02C0759567950A94E2F744
:100A90006170772786E0F8DE61E084E0F5DE60E0F3
:100AA00084E0F2DE219768F7DF91CF911F910F91DB
:100AB0000895CF93C82F60E087E0E6DE80E0D9DFBD
:100AC0008C2FD7DF61E087E0CF91DECE823059F006
:100AD00020F4813061F480E009C0833031F084304B
:100AE00031F484E103C083E001C08AE0E2CF80E01A
:100AF000E0DF81E08093790008951F920F920FB696
:100B00000F9211242F933F938F939F93AF93BF9393
:100B100080916D0090916E00A0916F00B091700077
:100B200030916C0020E3230F2D3720F44096A11D57
:100B3000B11D05C023EB230F4196A11DB11D2093CC
:100B40006C0080936D0090936E00A0936F00B09343
:100B500070008091710090917200A0917300B0912B
:100B600074000196A11DB11D8093710090937200D5
:100B7000A0937300B0937400BF91AF919F918F9138
:100B80003F912F910F900FBE0F901F901895789462
:100B900080B7826080BF80B7816080BF83B782608A
:100BA00083BF83B7816083BF89B7816089BF1EBC63
:100BB0008EB582608EBD8FB581608FBD3298319ABF
:100BC000309A379A1092750061E087E097DE61E015
:100BD00087E05ADE61E086E091DE60E086E054DE88
:100BE00061E084E08BDE61E084E04EDE61E083E082
:100BF00085DE60E083E048DE60E080E07FDE60E08C
:100C000081E07CDE60E082E079DE87E090E0DCD1AC
:100C1000C82F8093790082E0ADDE8536910544F0DF
:100C2000CF5FC0937900C53018F081E080937900E0
:100C300061E082E063DE61E082E026DE60917900BF
:100C40006093780087E090E0C7D1809179003EDF23
:100C500061E083E019DEC0E0D0E06091790080912E
:100C60007800681741F087E090E0B6D18091790074
:100C7000809378002BDF61E083E006DE64EF71E0B3
:100C800080E090E0BEDE81E075DE880F991FFC01F8
:100C9000E15BFF4FE590F49010917900E12FF0E0D7
:100CA000EE0FFF1FEF59FF4F808191818E159F0539
:100CB00094F501E00093760060E083E0E5DD68EC08
:100CC00070E080E090E09DDE61E083E0DDDD65E8DE
:100CD00070E080E090E095DE60E083E0D5DD68ECD8
:100CE00070E080E090E08DDE61E083E0CDDD65E8DE
:100CF00070E080E090E085DE60E083E0C5DD64EFD9
:100D000071E080E090E07DDE115019F010937900E1
:100D100002C00093790080917600882379F0E091F9
:100D20007900F0E0EE0FFF1FEF59FF4F80819181B6
:100D30000197E816F90614F41092760062E370E069
:100D400080E090E05EDE81E015DE880F991FFC01F7
:100D5000E15BFF4F85919491823491050CF46FC053
:100D600081E08093770060E083E08EDD60E083E0E7
:100D70008BDD68EC70E080E090E043DE61E083E0D2
:100D800083DD65E870E080E090E03BDE60E083E0DA
:100D90007BDD68EC70E080E090E033DE61E083E0D2
:100DA00073DD65E870E080E090E02BDE60E083E0DA
:100DB0006BDD68EC70E080E090E023DE61E083E0D2
:100DC00063DD65E870E080E090E01BDE60E083E0DA
:100DD0005BDD68EC70E080E090E013DE61E083E0D2
:100DE00053DD65E870E080E090E00BDE60E083E0DA
:100DF0004BDD64EF71E080E090E003DE68EC70E0D2
:100E000080E090E0FEDD81E0B5DD880F991FFC01F8
:100E1000E15BFF4F859194910196E0917900F0E0BC
:100E2000EE0FFF1FEF59FF4F20813181821793078B
:100E30002CF71092770061E083E026DDDFCF62E3DC
:100E400070E080E090E0DDDD80E094DD811522E05F
:100E500092070CF062C0809179008093780081E065
:100E60008093790061E087E090E0B6D080917900CE
:100E70002DDE60E083E008DD68EC70E080E090E06B
:100E8000C0DD61E083E000DD65E870E080E090E0D7
:100E9000B8DD60E083E0F8DC68EC70E080E090E0D2
:100EA000B0DD61E083E0F0DC65E870E080E090E0D8
:100EB000A8DD60E083E0E8DC68EC70E080E090E0D2
:100EC000A0DD61E083E0E0DC65E870E080E090E0D8
:100ED00098DD60E083E0D8DC68EC70E080E090E0D2
:100EE00090DD61E083E0D0DC65E870E080E090E0D8
:100EF00088DD60E083E0C8DC68EC70E080E090E0D2
:100F000080DD61E083E0C0DC65E870E080E090E0D7
:100F100078DD60E083E0B8DCFFCF8C319240DCF517
:100F200060E083E0B1DC68EC70E080E090E069DDD7
:100F300061E083E0A9DC65E870E080E090E061DDDD
:100F400060E083E0A1DC68EC70E080E090E059DDD7
:100F500061E083E099DC65E870E080E090E051DDDD
:100F600060E083E091DC68EC70E080E090E049DDD7
:100F700061E083E089DC65E870E080E090E041DDDD
:100F800060E083E081DC64EF71E080E090E039DDD7
:100F900081E08093790062E370E080E090E031DDF1
:100FA00080917900843059F480916000882339F071
:100FB0001092600068E873E180E090E022DD209705
:100FC00009F44BCE1DD849CEE199FECF9FBB8EBB15
:100FD000E09A99278DB30895262FE199FECF1CBA88
:100FE0009FBB8EBB2DBB0FB6F894E29AE19A0FBE61
:080FF00001960895F894FFCF6B
:0C0FF8000140003F003B003700320000C9
:00000001FF
